:100000000AC30FC30EC30DC30CC30BC30AC309C37A
:1000100008C307C306C305C304C303C302C301C3A4
:1000200000C3FFC2FEC269000000F5003C007B0077
:100030003C003D003C007B003C003D003C007B0060
:100040003C003D003C003D003C007B003C003D008E
:100050003C003D003C003D003C003D00C60AF6006F
:100060003C007B003C003D003C007B003C003D0030
:100070003C007B003C003D003C003D003C007B0020
:100080003C003D003C003D003C003D003C003D008C
:100090000000460000009B019A013400CD003400AE
:1000A000CD003400CD003400CD00340066003400B3
:1000B00066003400CD00340066003400CD0034000A
:1000C00066003400CD003400660034006600340061
:1000D000660034006600340066003400CD00340051
:1000E000CD00340066003400CD00340066003400DA
:1000F000CD00340066003400CD00340035039B0190
:100100009A013400CD003400CD003400CD0034001D
:10011000CD0034006600340066003400CD003400A9
:1001200066003400CD00340066003400CD00340099
:100130006600340066003400660034006600340057
:1001400066003400CD003400CD0034006600340079
:10015000CD00340066003400CD0034006600340069
:10016000CD00340000006D0000006601B3002C00DB
:100170002D002C0087002C002D002C002D002C00C1
:100180002D002C002D002C002D002C002D002C000B
:100190002D002C002D002C002D002C002D002C00FB
:1001A0002D002C0087002C002D002C002D002C0091
:1001B0002D002C002D002C002D002C002D002C00DB
:1001C0002D002C002D002C002D002C0087002C0071
:1001D0002D002C002D002C002D002C002D002C00BB
:1001E0002D002C002D002C002D002C002D002C00AB
:1001F00087002C002D002C0087002C0087002C008D
:1002000087002C0087002C002D002C002D002C00D6
:1002100087002C002D002C0087002C0087002C006C
:1002200087002C0087002C002D002C0087002C005C
:10023000281E6601B4002C002D002C0087002C0025
:100240002D002C002D002C002D002C002D002C004A
:100250002D002C002D002C002D002C002D002C003A
:100260002D002C002D002C002D002C0087002C00D0
:100270002D002C002D002C002D002C002D002C001A
:100280002D002C002D002C002D002C002D002C000A
:100290002D002C0087002C002D002C002D002C00A0
:1002A0002D002C002D002C002D002C002D002C00EA
:1002B0002D002C002D002C0087002C002D002C0080
:1002C00087002C0087002C0087002C0087002C0062
:1002D0002D002C002D002C0087002C002D002C0060
:1002E00087002C0087002C0087002C0087002C0042
:1002F0002D002C0087002C000000690000001C006D
:10030000BD001D0051001D0051001D0051001D00C9
:1003100051001D0051001D00BD001D00BD001D004D
:1003200051001D00BD001D0051001D0051001D00A9
:1003300051001D00BD001D0051001D003E121D009A
:10034000BD001D0051001D0051001D0051001D0089
:1003500051001D00BD001D0051001D0051001D0079
:10036000BD001D0051001D00BD001D00BD001D0091
:10037000BD001D0051001D00BD001D003E121D00EE
:10038000BD001D0051001D0051001D0051001D0049
:1003900051001D0051001D00BD001D00BD001D00CD
:1003A00051001D00BD001D0051001D0051001D0029
:1003B00051001D00BD001D0051001D003E121D001A
:1003C000BD001D0051001D0051001D0051001D0009
:1003D00051001D00BD001D0051001D0051001D00F9
:1003E000BD001D0051001D00BD001D00BD001D0011
:1003F000BD001D0051001D00BD001D000000690072
:1004000000009C03D0013A0039003A0039003A005C
:1004100039003A0039003A0039003A0039003A0010
:10042000AD003A0039003A00AD003A00AD003A00A4
:10043000AD003A00AD003A00AD003A00AD003A0020
:1004400039003A00AD003A0039003A00AD003A00F8
:1004500039003A0039003A00AD003A0039003A005C
:1004600039003A0039003A00AD003A0039003A004C
:10047000AD003A00AD003A0039003A00AD003A0054
:10048000AD003A00AD003A00D60F9E03E6003A00F8
:1004900098269E03E6003A000000710000005C0010
:1004A0005C00B8005C005C005C005C005C005C0010
:1004B0005C005C005C005C005C005C005C005C005C
:1004C000B8005C005C00B8005C005C0000245C00CC
:1004D0005C00B8005C005C005C005C005C005C00E0
:1004E0005C005C005C005C005C005C005C005C002C
:1004F000B8005C005C00B8005C005C0000006900B3
:100500000000CE01DC013500AF003500AF00350042
:10051000AF0035003E0035003E0035003E0035009E
:100520003E0035003E003500AF003500AF0035001D
:10053000AF0035003E0035003E0035003E0035007E
:100540003E0035003E0035003E003500AF0035006E
:100550003E0035003E0035003E0035003E003500CF
:100560003E0035003E003500AF0035003E0035004E
:10057000AF003500AF003500AF003500AF003500EB
:10058000AF003500AF0035003512D001DC01350079
:10059000AF003500AF003500AF0035003E0035003C
:1005A0003E0035003E0035003E0035003E0035007F
:1005B000AF003500AF003500AF0035003E0035001C
:1005C0003E0035003E0035003E0035003E0035005F
:1005D0003E003500AF0035003E0035003E003500DE
:1005E0003E0035003E0035003E0035003E0035003F
:1005F000AF0035003E003500AF003500AF003500DC
:10060000AF003500AF003500AF003500AF0035005A
:1006100000000000000011241FBECFEDCDBF5FD051
:10062000A7C0EECC0CC020E030E0809A2F5F3F4F97
:1006300027303105D1F761507040804090406115FE
:1006400071058105910579F70895C09A68EB7BE003
:1006500080E090E0E7DFC0980895F7DF68E97AE38B
:1006600080E090E0DFDFF1DF68E97AE380E090E0AE
:10067000D9DFEBDF68E97AE380E090E0D3DFE5DF04
:100680000895EF92FF920F931F938C0182E480BF35
:1006900081E083BF000F111F000F111F96E2E92EAA
:1006A00090E0F92EF701E00FF11F6591749180E061
:1006B00090E0B8DF83B7887F83BF80B78F7380BF38
:1006C000C298F8013296EE0DFF1D6591749180E09D
:1006D00090E0A8DF1F910F91FF90EF9008950F9386
:1006E0001F93CF93DF9319BE8FEF87BB18BAC0E07B
:1006F000D0E016C0AADF06BF2196CE01C2DFFE0100
:10070000EE0FFF1FEE0FFF1FE85DFF4F85919491E5
:10071000892B91F768EA71E680E090E083DF21960B
:10072000FE01EE0FFF1FEE0FFF1FEA5DFF4F059169
:10073000149101151105F1F690DF83B7887F83BF0F
:1007400080B78F7380BF85B7806285BF85B78061B2
:1007500085BF68EE73E080E090E064DF18BA17BAF6
:10076000889580E090E0DF91CF911F910F910895DF
:04077000F894FFCF2B
:00000001FF
